:020000040800F2
:10000000200E002439030008890A0090BB090090E3
:1000100045030008790000900F16009000000000D2
:100020000000000000000000000000008D0A0090A9
:100030007B000090000000008B0A00908F0A009067
:100040005303000853030008530300085303000838
:100050005303000853030008530300085303000828
:100060005303000853030008530300085303000818
:100070005303000853030008530300085303000808
:1000800053030008530300085303000853030008F8
:1000900053030008530300085303000853030008E8
:1000A00053030008530300085303000853030008D8
:1000B00053030008950A00905303000853030008F7
:1000C00053030008530300085303000853030008B8
:1000D0005303000879140008530300085303000871
:1000E00053030008530300080000000053030008F6
:1000F0005303000853030008530300085303000888
:100100005303000853030008530300085303000877
:100110005303000853030008530300085303000867
:100120005303000853030008530300085303000857
:100130005303000853030008530300085303000847
:1001400000000000000000000000000000000000AF
:100150005303000853030008530300085303000827
:100160005303000853030008530300085303000817
:100170005303000853030008530300085303000807
:1001800053030008530300085303000853030008F7
:1001900053030008530300085303000853030008E7
:1001A00053030008530300085303000853030008D7
:1001B00053030008530300085303000853030008C7
:1001C00053030008530300085303000853030008B7
:1001D00053030008530300085303000853030008A7
:1001E0005303000853030008530300085303000897
:1001F0005303000853030008530300085303000887
:100200005303000853030008530300085303000876
:100210005303000853030008530300085303000866
:1002200053030008530300085303000800000000B4
:1002300053030008530300080000000053030008A4
:100240005303000853030008530300085303000836
:100250005303000853030008530300085303000826
:100260005303000853030008530300085303000816
:100270005303000853030008530300080000000064
:1002800053030008000000005303000800000000B2
:10029000000000005303000800F002F800F03CF8F2
:1002A0000AA090E8000C82448344AAF10107DA45D1
:1002B00001D100F031F8AFF2090EBAE80F0013F0E7
:1002C000010F18BFFB1A43F0010318472C1300005D
:1002D0004C130000103A24BF78C878C1FAD85207EE
:1002E00024BF30C830C144BF04680C6070470000B0
:1002F0000023002400250026103A28BF78C1FBD82F
:10030000520728BF30C148BF0B6070471FB501F0CE
:1003100065F91FBD10B510BD00F0AAF81146FFF732
:10032000F5FF01F00FF900F0C8F803B4FFF7F2FF92
:1003300003BC01F0D3F80000094880470948004792
:10034000FEE7FEE7FEE7FEE7FEE7FEE7FEE7FEE785
:10035000FEE7FEE704480549054A064B70470000E2
:10036000F51300089902000820020024200E002442
:100370002004002420040024704753EA020C00F0FB
:1003800069802DE9F04B4FF00006002B1FBFB3FA38
:1003900083F503FA05F424FA05F65E4012BF16430E
:1003A000B2FA82F502FA05F4C5F120051EBF22FA61
:1003B00005FC44EA0C04203556EA044C4FEA144488
:1003C00018BF641C4FF000084FF00009904271EB19
:1003D000030C39D3002919BFB1FA81F701FA07F6E6
:1003E000B0FA80F700FA07F6C7F120071EBF20FA1F
:1003F00007FC46EA0C062037B6FBF4FCA7EB050722
:10040000103F07F01F0BCBF120060CFA0BFB2CFA68
:1004100006F644BFB3460026202FA4BF5E464FF029
:10042000000B5BEA060C08BF4FF0010B19EB0B0940
:10043000ABFB027C48EB0608C01B06FB02CC0BFBA7
:1004400003CC71EB0C01C1E70B460246414648461E
:10045000BDE8F08B13B54FF000004FF00001AFF393
:100460000080BDE81C407047704770477047704778
:10047000754600F02BF8AE4605006946534620F05D
:100480000700854618B020B5FFF764FFBDE820409F
:100490004FF000064FF000074FF000084FF0000B40
:1004A00021F00701AC46ACE8C009ACE8C009ACE8F3
:1004B000C009ACE8C0098D46704710B50446AFF3DB
:1004C00000802046BDE81040FFF72FBF004870476E
:1004D000C001002440F2111CC9F2000C604740F238
:1004E000297CC9F2000C604740F21B7CC9F2000C69
:1004F000604740F6131CC9F2000C604740F63D2CE3
:10050000C9F2000C604740F6BD1CC9F2000C604700
:1005100040F6A12CC9F2000C604740F6B96CC9F254
:10052000000C604740F6A90CC9F2000C60470000BF
:10053000F0B5BFF34F8FBFF36F8F1D4900200860E8
:10054000BFF34F8FBFF36F8F1A4C216841F4003116
:100550002160BFF34F8FBFF36F8F16497031086072
:10056000BFF34F8F081F006843F6FF75104E10361B
:10057000C0F34E31C0F3C90305EA4112184642EAFE
:1005800080773760401EFAD2491EF5D2BFF34F8FF5
:10059000206840F480302060BFF34F8FBFF36F8F2F
:1005A00003484C30016841F004010160F0BD0000D7
:1005B00050EF00E014ED00E00248016841F0010155
:1005C00001607047200400582DE9F84F6C4C002260
:1005D0004FF0B04A4FF0010B4FF0030E4FF00F09F0
:1005E0000B680BFA02F73B40BB4270D14D68022DFD
:1005F00001D0122D12D1D50800EB850CDCF820605B
:100600005507ED0E09FA05F826EA0806D1F810801C
:1006100008FA05F848EA0608CCF82080D0F80080EF
:10062000560091F804C00EFA06F50CF0030C28EA07
:1006300005080CFA06FC4CEA080CC0F800C0D1F81A
:1006400004C0BCF1010F08D0BCF1020F05D0BCF111
:10065000110F02D0BCF1120F16D1D0F808C0D1F89A
:100660000C802CEA050C08FA06F848EA0C08C0F8D9
:100670000880D0F804C02CEA070C0F79C7F30017E4
:10068000974047EA0C074760C768AF438D68B5409D
:100690003D43C5604D68ED006BD53A4D2E6846F080
:1006A00002062E602D6822F0030606F1B04605F022
:1006B00002050095D6F808C495072F0F09FA07F52B
:1006C0002CEA050C304DA84202D100252EE050E066
:1006D0002E4DA84201D1012528E02D4DA84201D17F
:1006E000022523E02B4DA84201D103251EE02A4D0F
:1006F000A84201D1042519E0284DA84201D10525C1
:1007000014E0274DA84201D106250FE0254DA8424F
:1007100001D107250AE0244DA84201D1082505E0B2
:10072000224DA84201D1092500E00A25BD4045EA35
:100730000C05C6F8085425684E689D43F60300D59D
:100740001D43256065684E689D43B60300D51D4373
:100750006560DAF8005056464F689D43FF0200D5A9
:100760001D43356075684F689D43BF0200D51D432A
:100770007560521C102AFFF433AFBDE8F88F0000FB
:1007800080000058F4440258000002580004025847
:1007900000080258000C02580010025800140258B9
:1007A00000180258001C0258002002580024025869
:1007B00042694A40426170470AB1018370474183F0
:1007C0007047000001488068704700001000002456
:1007D000024881680278114481607047100000244B
:1007E000032010B500F058F80F2000F007F808B10A
:1007F000012010BD00F022F8002010BD70B50D4D95
:1008000004464FF47A712878B1FBF0F00A49096880
:10081000B1FBF0F000F05AFC48B9102C07D20022CE
:100820002146501E00F018F800206C6070BD0120B9
:1008300070BD000010000024000000247047002854
:1008400009DB012100F01F0291404009800000F106
:10085000E020C0F8001170470E4BF0B41B68C3F3E2
:100860000223C3F10704042C00D904241D1D072D05
:1008700001D2002300E0DB1E012606FA04F56D1EFE
:100880000D409D409E40761E164045EA0601F0BC94
:1008900000F014BE0CED00E0064A00F007011068FD
:1008A0004FF6FF03184040EA012003490843106057
:1008B000704700000CED00E00000FA052DE9F0475C
:1008C000DFF8BC9104460E46D9F8000000F007009E
:1008D000B0420CD2D9F8001021F007013143C9F819
:1008E0000010D9F8000000F00700B0427ED1207857
:1008F000DFF89081800707D5D8F80010E26821F072
:100900000F011143C8F800102078C00762D0D8F852
:100910000010A26821F470611143C8F80010594911
:100920006068183902281CD003281DD009680128E6
:100930001DD04907002960DA524F083F396821F07D
:10094000070101433960FFF73DFF0546606841F24A
:100950008831022813D003281ED001288A4627D0C8
:1009600034E009688903E5E709688901E2E7C90518
:10097000E0E7FFF727FF411B514501D923E08A46F5
:100980003868C0F3C2000228F3D123E0FFF71AFF52
:10099000411B514501D916E08A463868C0F3C200B0
:1009A0000328F3D116E0FFF70DFF411B51450AD88C
:1009B0003868C0F3C2000128F5D10BE0FFF702FF51
:1009C000411B514502D90320BDE8F087386810F07B
:1009D000380FF3D1D9F80010484601F00701B142B1
:1009E0000DD9016821F00701314300E005E0016005
:1009F000006800F00700B04201D00120E4E7207851
:100A0000400707D5D8F80010226921F07001114382
:100A1000C8F80010207801071B4805D501686269F5
:100A200021F07001114301602178C90605D50168E4
:100A3000A26921F4E061114301602078800607D5A6
:100A40001149091D0868E26920F070001043086030
:100A500000F066F8D8F800104FF4807292FAA2F213
:100A600001F47061B2FA82F2D140084A515CC84088
:100A7000074908600F20FFF7C1FE0020A4E700002F
:100A800000200052184402581C440258E615000881
:100A90000000002410B5FFF71DFD08490968012278
:100AA00092FAA2F201F00F01B2FA82F2D140044AA6
:100AB000515CC8400349086010BD0000184402584A
:100AC000E61500080400002410B5FFF7E3FF07490E
:100AD0000968102292FAA2F201F07001B2FA82F2D1
:100AE000D140034A515CC84010BD00001C4402586C
:100AF000E615000810B5FFF7CDFF074909684FF468
:100B0000807292FAA2F201F4E061B2FA82F2D1406C
:100B1000024A515CC84010BD1C440258E61500084A
:100B20003548F0B50068364D10F03801334809D02B
:100B30000411082904D0334E10290BD018290BD0EA
:100B40002046F0BD29688906FBD52968C1F3C1019B
:100B5000C840F0BD3046F0BD274918310A68096821
:100B600012F00302284BC1F305111B68274F03F055
:100B700001033F68DFED260AB7EE001AC7F3CC0782
:100B800017FB03F300EE103A224BB8EE400A06D0F2
:100B9000012A01D0022A2BD0B4FBF1F008E02A6828
:100BA000920603D52A68C2F3C102D040B0FBF1F02F
:100BB00001EE900A1868B8EE612AC0F3080001EE51
:100BC000900A1868F8EE611A40EE201A31EE810A98
:100BD00022EE000AC0F34620401C00EE900AF8EE18
:100BE000600A80EE201ABCEEC10A10EE100AF0BDB9
:100BF000B6FBF1F0DCE70000104402580090D0038F
:100C00000044025840787D012C4402583444025874
:100C100000000039304402582DE9F05F04460078A6
:100C2000DFF8FC8341F28839DFF8F8A3FE4DC007F6
:100C30004ED0D8F800104046C1F3C20102291AD0A4
:100C40000068C0F3C200032805D1DAF8000000F004
:100C5000030002280FD06068B0F5803F12D010B1B9
:100C6000B0F5A02F19D0286820F4803028602868BB
:100C700020F4802009E02868800329D560680028D6
:100C800074D025E0286840F480302860606890B116
:100C9000FFF798FD06464F4609E0286840F480209B
:100CA0002860EFE7FFF78EFD801BB8427DD82868EB
:100CB0008003F7D50CE0FFF785FD06464F4604E0BC
:100CC000FFF780FD801BB842F0D828688003F7D476
:100CD0002078D64F80075AD5D8F8001040464FF4F8
:100CE0007C3B11F0380F13D00068C0F3C20003281A
:100CF00003D1DAF8000080070AD0E068A8B32968B9
:100D000021F0190101432960FFF75CFD06461DE053
:100D10002868400702D5E0680028B1D02868E1685B
:100D200020F0190008432860FFF74CFD064604E058
:100D3000FFF748FD801B0228B8D828684007F7D580
:100D400007E0FFF73FFD801B0228AFD82868400767
:100D5000F7D538689BFAABF220F47C312069B2FAFF
:100D600082F290400143396011E000E0AEE0286873
:100D700020F001002860FFF725FD064604E0FFF79C
:100D800021FD801B022891D828684007F7D42078DD
:100D9000C00655D5D8F8001040464FF0F84BC1F3C7
:100DA000C201012917D0006800E0EDE0C0F3C200E5
:100DB000032805D1DAF8000000F0030001280AD06A
:100DC000E069002828682CD040F080002860FFF7F8
:100DD000F9FC064616E02868C00502D5E0698028BF
:100DE00074D138689BFAABF220F0F841206AB2FA6D
:100DF00082F290400143396022E0FFF7E3FC801B60
:100E0000022899D82868C005F7D538689BFAABF254
:100E1000216AB2FA82F220F0F8409140084338602B
:100E20000EE020F080002860FFF7CCFC064604E0CE
:100E3000FFF7C8FC801B022887D82868C005F7D4B4
:100E40002078000724D5774F60694C370028386830
:100E50000FD040F001003860FFF7B4FC064604E014
:100E6000FFF7B0FC801B02288DD838688007F7D5C3
:100E70000EE020F001003860FFF7A4FC064604E015
:100E8000FFF7A0FC801B02287ED838688007F7D4C3
:100E90002078800623D5A069002828680FD040F468
:100EA00080502860FFF78EFC064604E0FFF78AFCBE
:100EB000801B022868D828688004F7D50FE020F44A
:100EC00080502860FFF77EFC064605E0D6E0FFF77D
:100ED00079FC801B022857D828688004F7D4207832
:100EE000400744D5524F386840F480703860FFF7AF
:100EF00069FC064604E0FFF765FC801B642843D8C4
:100F00003868C005F7D5474FA068483701280AD090
:100F100008B1052811D0386820F001003860386821
:100F200020F0040002E0386840F001003860A0685A
:100F300088B1FFF747FC064609E0386840F0040036
:100F40003860F0E7FFF73EFC811B49451CD8386844
:100F50008007F7D50BE0FFF735FC064604E0FFF706
:100F600031FC811B49450FD838688007F7D4606A87
:100F7000F0B3D8F80010C1F3C20103297ED00228D3
:100F8000286820F0807000E079E0286003D0FFF747
:100F900019FC044687E0FFF715FC064604E0FFF75E
:100FA00011FC801B02287BD828688001F7D4DAF86E
:100FB000001040F2F3329143E26A41EA0211A26A60
:100FC0001143CAF8001094F834004FF4FE02218E49
:100FD0004002491EA0F5007080B2C1F30801084329
:100FE000218F491E02EA0141084394F83C1000E0B9
:100FF0005CE0491E120202EA016108430949083116
:1010000008600B1D19684FF6F872A06C914392FAB4
:10101000A2F2B2FA82F2904001431960014809E05D
:10102000104402582844025800440258044402580C
:1010300000480258001D0168226C21F00C01114388
:1010400001600168626C21F00201114301600168D6
:1010500041F480310160016841F4003101600168B0
:1010600041F480210160016841F0010101602868BC
:1010700040F080702860FFF7A5FB01E018E00FE06A
:10108000044604E0FFF79EFB001B022808D82868EE
:101090008001F7D50AE0FFF795FB001B022802D973
:1010A0000320BDE8F09F28688001F4D40020F8E711
:1010B0000120F6E74FF0E0210428086903D020F072
:1010C00004000861704740F00400FAE7401EB0F1E8
:1010D000807F10B501D3012010BD4FF0E024606186
:1010E0000F21601700F0EAF90020A06107202061BD
:1010F000002010BD10B5006886B01B49884230D171
:101100001A48016841F001010160006800F0010027
:10111000059016481030016841F010010160006828
:101120000121134C00F0100005904FF40070009066
:101130000220CDE901010390072069460490204672
:10114000FFF742FA4FF48061204600916946FFF7AD
:101150003BFA2520FFF773FB032225201146FFF7FA
:101160007BFB06B010BD000000100140E0440258B7
:101170000000025830B50068114988420CD1114A6C
:101180005088010408D411464FF000034404097844
:1011900006D50A2901D0538030BD40F400400DE04F
:1011A0000D2909D0084DC0F30D04401C80B2C7289A
:1011B00029555080EFD830BD40F48040508030BD7C
:1011C000001001400C0000241C00002454482DE9AC
:1011D000F041524C86B0016841F0020101600168A3
:1011E00041F0200101604E480C38016841F4804113
:1011F000016040200090022001900320DFF824814C
:10120000002569460A270497CDE902504046FFF7BA
:10121000DBF9042069460926049600904046FFF752
:10122000D3F90496C020404E694600903046FFF73F
:10123000CBF94FF440706946049700903046FFF7B1
:10124000C3F937486438016841F48041016001689E
:1012500021F4804101603148203881688906FCD43E
:101260003249016032494160016841F00101016089
:1012700081688906FCD44FF49C71416181688907BB
:10128000FCD5C16841F00201C16081688906FCD4C7
:101290004FF48371416181688907FCD5C16841F0D1
:1012A0000201C16081688906FCD42249416105615F
:1012B00081684907FCD530212170016841F00401A3
:1012C000016081688907FCD5C16841F00201C160F5
:1012D00081688906FCD481688906FCD4C5611649F9
:1012E00041611648016821F4803101601349703171
:1012F0000A6822F001020A600A1D156082060F4B7F
:1013000078331A601B1D0E4A1A6005220A600168B4
:1013100041F48031016006B0BDE8F08120500052F8
:10132000E04402580004025800140258100300015F
:1013300001041600C0030003EBEF180F24ED00E0DA
:101340002D00030370B5294C9CB0256825F00405D9
:101350002560264C00260C34256845F44045256060
:10136000256805F440451B952568AD04FCD501248E
:1013700000940CAD03962404019402240994CDE951
:101380000A410796082485E80D00CDE91046684615
:10139000FFF742FC98B9FFF719FF3F201390032095
:1013A000CDE9140640200101CDE91640CDE9180130
:1013B00050201A90022113A8FFF780FA10B10120E3
:1013C0001CB070BD0A48016841F080010160084806
:1013D000F430016841F002010160006800F0020091
:1013E0001B90FFF7E9F80020EAE700000C480258DC
:1013F000004402581C48016841F4700101601B4917
:10140000086840F001000860184A0020103210609F
:101410000A68174B1A400A60144A18321060121DED
:101420001060121D1060114A28321060121D1060E9
:10143000121D1060121D1060121D1060121D106030
:10144000121D1060121D10600A6822F480220A60CA
:1014500006496031086001200649C1F80801C0064C
:10146000014980390860704788ED00E00044025867
:101470007FEDF6EA0080005170B50D4D00240D4857
:10148000FFF72DF802E0641CAC4204D80948FFF7CE
:101490002BF82028F7D1002402E0641CAC4206D8C7
:1014A000054901220348FFF724F80028F5D170BD53
:1014B000FFFF0100E40000240C0000240907090ECE
:1014C000002804DB00F1E02080F80014704700F0F1
:1014D0000F0000F1E02080F8141D704770470000F5
:1014E00010B504460420FFF7E5FD0148046010BD77
:1014F0000800002470B5002405464FF47A7603E016
:10150000304600F005F8641CAC42F9D370BD000011
:1015100070B54FF0E02500216C69094AAB6912688B
:101520005043AA699A42FCD002D2A3EB020302E024
:10153000A4EB02063344194413468142F1D370BD33
:101540000800002401250024FEF7F2FFFFF748F908
:10155000042302220521A020FFF7F4FE4FF4C870F7
:10156000FFF7BEFF4FF4E13000F01CF8FEF7C6FFB6
:10157000FEF7C9FFC72140F2F310FEF7C9FF4FF491
:1015800096760A20FFF7B6FF0DB1641C00E0641EDA
:10159000A4B2B44200D9002504B901252046FEF7C3
:1015A000BCFFEEE70B490A4A10B5C1E90020002054
:1015B0008860C860086188610C2048610846FEF7B1
:1015C000B1FFBDE81040044901220248FEF791BF77
:1015D00000100140E40000240C0000244FF0407093
:1015E000E1EE100A7047000000000102030401024E
:1015F000030406070809000018160008000000246C
:101600001C000000D4020008341600081C0000244E
:10161000040E0000F00200080090D0030090D003F8
:1016200000000000000000000100000010000000A9
:0416300000000000B6
:0200000490006A
:1000000040F6213CC0F6000C604740F6952CC0F647
:10001000000C604740F2C95CC0F6000C604740F23B
:10002000B17CC0F6000C604741F2F50CC0F6000C44
:10003000604740F2B97CC0F6000C604740F2D17CCA
:10004000C0F6000C604740F2C57CC0F6000C60476B
:1000500041F2751CC0F6000C604740F27B3CC0F6D4
:10006000000C604740F6C92CC0F6000C604740F613
:10007000F52CC0F6000C6047FEE7704710B528B1BC
:1000800090F83510022903D080214165012010BD70
:100090001D4A4FF4956301688C189C4207D80422CE
:1000A00080F83520086820F00100086029E00C681D
:1000B00024F00E040C6001680A440A6822F0010270
:1000C0000A60016E0A6822F480720A6090F85C305F
:1000D000012202FA03F10D4B1960D0E919134B60AC
:1000E000C16E31B10B6823F480730B60D0E91C132F
:1000F0004B60002180F8341080F83520016D01B18B
:100100008847002010BD0000F0FFFDBF04540258D6
:1001100010B5FFF775FF084909684FF4807292FA2D
:10012000A2F201F47061B2FA82F2D140034A515C4A
:10013000C8400349086010BD18440258E61500087D
:100140000000002410B5FFF760FF0749096810227E
:1001500092FAA2F201F07001B2FA82F2D140034A9F
:10016000515CC84010BD000020440258E61500084C
:10017000364930B50A68096812F00302344BC1F3FE
:1001800005311B68334C03F010032468DFED320A9D
:10019000B7EE001AC4F3CC0414FB03F300EE103ADC
:1001A0002E4BB8EE400A07D02D4C012A01D0022A6E
:1001B0004AD0B4FBF1F10BE0244C283C22689506B0
:1001C000284A03D52468C4F3C104E240B2FBF1F12C
:1001D00001EE901A1968B8EE612AC1F3080101EE28
:1001E000901A1968F8EE611A40EE201A31EE810A71
:1001F00022EE000AC1F34621491C00EE901AF8EEE7
:10020000600A80EE201AFCEEC10AC0ED000A1968EF
:10021000C1F30641491C00EE901AF8EE600A80EE28
:10022000201AFCEEC10AC0ED010A1968C1F306618B
:10023000491C00EE901AF8EE600A80EE201ABCEE1F
:10024000C10A80ED020A30BD074ABFE728440258C0
:100250002C4402583C4402580000003938440258EB
:1002600000093D000090D00340787D01364930B54B
:100270000A68096812F00302344BC1F305511B6888
:10028000334C03F480732468DFED320AB7EE001AB2
:10029000C4F3CC0414FB03F300EE103A2E4BB8EE7B
:1002A000400A07D02D4C012A01D0022A4AD0B4FBC3
:1002B000F1F10BE0244C283C22689506284A03D52E
:1002C0002468C4F3C104E240B2FBF1F101EE901ADC
:1002D0001968B8EE612AC1F3080101EE901A196895
:1002E000F8EE611A40EE201A31EE810A22EE000A81
:1002F000C1F34621491C00EE901AF8EE600A80EE28
:10030000201AFCEEC10AC0ED000A1968C1F30641CB
:10031000491C00EE901AF8EE600A80EE201AFCEEFE
:10032000C10AC0ED010A1968C1F30661491C00EE5B
:10033000901AF8EE600A80EE201ABCEEC10A80ED39
:10034000020A30BD074ABFE7284402582C4402582D
:1003500044440258000000394044025800093D005E
:100360000090D00340787D0170477047704770B5AA
:100370000446006801694FF00005C943890715D498
:10038000C168C943890711D4E91E016101202077A2
:10039000206880698007204602D0FFF7E7FF04E06D
:1003A00000F0A5F8204600F07BF925772068016968
:1003B000C943490717D4C168C943490713D46FF02B
:1003C00004010161022020772068806910F4407FD9
:1003D000204602D0FFF7CAFF04E000F088F820466C
:1003E00000F05EF9257720680169C943090716D432
:1003F000C168C943090712D46FF0080101610420E4
:1004000020772068C0698007204602D0FFF7AEFF42
:1004100004E000F06CF8204600F042F925772068EF
:100420000169C943C90617D4C168C943C90613D4B1
:100430006FF010010161082020772068C06910F476
:10044000407F204602D0FFF791FF04E000F04FF814
:10045000204600F025F9257720680169C943C907BE
:1004600008D1C168C943C90704D1891E016120466A
:1004700000F044F9206801696FF08005C94309065E
:1004800007D4C168C943090603D405612046FFF7B4
:100490006BFF20680169C943C90507D4C168C94316
:1004A000090603D405612046FFF75EFF2068016955
:1004B000C943490609D4C168C943490605D46FF048
:1004C00040010161204600F025F920680169C94317
:1004D00089060BD4C168C943890607D46FF020018F
:1004E00001612046BDE87040FFF73FBF70BD704717
:1004F00070B5044690F83C000D4601280ED0012648
:1005000084F83C60022084F83D000C2A45D007DCCA
:100510005AB1042A1BD0082A78D12CE0022070BDE1
:10052000102A4ED0142A71D15DE0206800F048FBFB
:100530002068816941F0080181612068816921F0AA
:1005400004018161206881692A69114311E02068F2
:1005500000F084FB2068816941F4006181612068BA
:10056000816921F480618161206881692A6941EA99
:10057000022181614AE0206800F0B8FB2068C1696F
:1005800041F00801C1612068C16921F00401C16125
:100590002068C1692A69114311E0206800F0EAFB74
:1005A0002068C16941F40061C1612068C16921F41A
:1005B0008061C1612068C1692A6941EA0221C16183
:1005C00024E0206800F00CFC2068416D41F0080137
:1005D00041652068416D21F0040141652068416D4D
:1005E0002A69114311E0206800F030FC2068416D59
:1005F00041F4006141652068416D21F480614165ED
:100600002068416D2A6941EA0221416584F83D6014
:10061000002084F83C0070BD10B5040003D094F8AD
:100620003D0010B107E0012010BD002084F83C001F
:10063000204600F00DF8022084F83D002068211DBE
:1006400000F052FA012084F83D00002010BD0000A7
:10065000114800B587B0016841F0020101600068EF
:1006600000F0020005900C480838016841F00201D2
:1006700001600068012100F0020005900220009056
:10068000CDE901010321CDE9031004486946FFF7D4
:10069000C1FC07B000BD0000E84402580004025845
:1006A0007047000010B501220446006800F07CFA93
:1006B0000D48216881420BD00C48814208D00C487B
:1006C000814205D00B48814202D00B48814203D1C0
:1006D000486C40F4004048642068018841F0010102
:1006E0000180002010BD0000000001400004014016
:1006F0000040014000440140004801400349884255
:1007000003D103480121FFF78ABC7047640100242C
:100710000004025870477047704790F8791090F8BD
:100720007A0008437047000070B502680446D0693B
:100730001368916810F00F0F64D0594D03F4907650
:100740000D40354376D0C50707D0DD0505D5012519
:100750001562E26F42F00102E267820708D5CA071C
:1007600006D0256802222A62E26F42F00402E267A4
:10077000420708D5CA0706D0256804222A62E26F1C
:1007800042F00202E26702070ED503F0200201F0F8
:1007900080552A4352EAC17206D0256808222A628F
:1007A000E26F42F00802E267E26F002A3AD0800668
:1007B00008D503F0200001F08051084302D0204604
:1007C00000F02AFCE06F000703D420688068400630
:1007D0002AD5204600F012FC2068816849061ED503
:1007E000816821F040018160606FC0B12D490165D1
:1007F000606FFFF743FC002814D0606F016DBDE807
:1008000070400847850615D503F0200501F0805695
:1008100035430FD02046BDE8704000F0FDBB2046B8
:10082000FFF77AFF70BD05E02046FFF775FF002057
:10083000E067F7E7C6024FF020050CD54E020AD557
:10084000E803106284F8795084F87A502046BDE8B5
:100850007040FFF760BF06060AD503F0800601F47A
:1008600000010E4304D02046BDE8704000F064BE95
:1008700041060BD5590609D51168204621F04001E3
:10088000116084F8795000F097F8CBE70002C9D5E1
:100890005800C7D5106820F080401060C2E7000003
:1008A00001000010E90F009010B5040003D094F887
:1008B000790010B107E0012010BD002084F8780015
:1008C0002046FFF7B1FB242084F8790020680168F6
:1008D00021F001010160204600F0DAFB0128EBD095
:1008E000606B10B1204600F0EDFA2068416821F4F9
:1008F000904141602068816821F02A018160206870
:10090000016841F0010101602046BDE8104000F09F
:100910003DBB90F87A30202B4CD1B9B1B2B190F8F0
:100920007830012B46D0012380F878304166A0F85A
:100930006820A0F86A20FF228168B1F5805F07D0A7
:100940007F2351B1B1F1805F0CD010E001207047DE
:10095000016921B940F2FF1107E0016909BBA0F864
:100960006C2004E00169E1B13F21A0F86C10002186
:10097000C167222280F87A2080F8781001688A689E
:1009800042F001028A6001680A6892000CD50A6888
:1009900042F480720A600068816841F08051816091
:1009A00006E0A0F86C30E2E7086840F49070086058
:1009B00000207047022070477047FEE71B4870B563
:1009C00086B0016841F001010160016801F0010198
:1009D0000591016841F004010160016801F0040122
:1009E0000591016841F08001016000680324002541
:1009F000694600F08000059002200126CDE902043E
:100A00000B48CDE90065FFF705FB700303948DE803
:100A1000610008486946FFF7FDFA0C20009006487F
:100A20006946FFF7F7FA06B070BD0000E0440258CF
:100A30000000025800080258001C0258104810B567
:100A400086B0016841F002010160006801210D4C8F
:100A500000F0020005900320CDE90001CDE902106D
:100A600069462046FFF7D6FA012220461146FFF7D5
:100A7000E0FA012220460221FFF7DBFA06B010BDA2
:100A8000E044025800040258704770477047FFF76F
:100A9000D5BA00000148FFF76ABC000064010024D9
:100AA000104A10B504460E48C2E900010020C2E910
:100AB000020410611046FFF7AFFD0A4960200C22C6
:100AC0004031086060084860022088600548FFF7F0
:100AD0000FFDBDE8104003480C21FFF7E3BD000007
:100AE00000040040640100242DE9F04702884FF023
:100AF000804A254C254D264EA042264F264B09D034
:100B0000504507D0A84205D0B04203D0B84201D02A
:100B1000984204D122F0700C4A6842EA0C02DFF8D5
:100B20007CC0DFF87C80A042DFF878900FD0504581
:100B30000DD0A8420BD0B04209D0B84207D098429D
:100B400005D0604503D0404501D0484503D122F48B
:100B50004075CA682A438D8A22F080022A430280A7
:100B60008A68C2620A880285A04207D0984205D0EE
:100B7000604503D0404501D0484501D1098A01862E
:100B800001214161BDE8F087000001400004004000
:100B900000080040000C00400004014000400140FB
:100BA0000044014000480140012310B5046A8B4015
:100BB0009C430462036A8A401343036210BD000031
:100BC0002DE9F043026A22F001020262056A4268DE
:100BD000836925F002051B4C1C4E23400C6823F052
:100BE00003031B4F1C438B68DFF868C02B43164D73
:100BF000DFF86490A84207D0B04205D0B84203D0D5
:100C0000604501D0484506D123F00808CB6843EA87
:100C1000080323F00403A84207D0B04205D0B8422D
:100C200003D0604501D0484505D14D6922F440729A
:100C300015438A692A4342608461496841630362BB
:100C4000BDE8F0838FFFFEFF00000140000401407B
:100C5000004001400044014000480140F0B5026AF4
:100C600022F010020262056A42688369194C1B4E29
:100C700023400C6823F4407343EA042425F0200346
:100C80008D6843EA0513144DA84201D0B04206D145
:100C9000CF6823F0800343EA071323F04003A84200
:100CA0000AD0B04208D00E4DA84205D00D4DA84242
:100CB00002D00D4DA84207D14D6922F4406242EAAC
:100CC00085028D6942EA85024260846149688163D8
:100CD0000362F0BDFF8FFFFE0000014000040140F1
:100CE000004001400044014000480140F0B5026A64
:100CF00022F480720262026A4368C46922F40072BC
:100D0000184E24F073050C682C438D6842EA0522C6
:100D1000134DA84201D0B04206D1CF6822F4006240
:100D200042EA072222F48062A8420AD0B04208D0E8
:100D30000D4DA84205D00D4DA84202D00C4DA84241
:100D400007D14D6923F4405343EA05138D6943EA03
:100D500005134360C4614968C1630262F0BD0000CD
:100D600000000140000401400040014000440140F7
:100D70000048014030B5026A22F480520262036AE0
:100D80004268C46923F400530D6824F4E64444EA3D
:100D900005248D6843EA05330C4DA8420BD00C4D59
:100DA000A84208D00B4DA84205D00B4DA84202D056
:100DB0000A4DA84204D14D6922F4804242EA8512CC
:100DC0004260C46149680164036230BD00000140B3
:100DD000000401400040014000440140004801403F
:100DE00030B5026A22F480320262046A4268436DBE
:100DF00024F4003423F070050B682B430D8944EA7A
:100E000005440D4DA8420BD00C4DA84208D00C4D06
:100E1000A84205D00B4DA84202D00B4DA84204D1E8
:100E20004D6922F4803242EA0522426043654968F6
:100E30008165046230BD00000000014000040140F3
:100E400000400140004401400048014030B5026AC2
:100E500022F480120262046A4268436D24F4001492
:100E60000D6823F4E04343EA05230D8944EA055461
:100E70000C4DA8420BD00C4DA84208D00B4DA842F7
:100E800005D00B4DA84202D00A4DA84204D14D69AD
:100E900022F4003242EA8522426043654968C16516
:100EA000046230BD000001400004014000400140E8
:100EB00000440140004801400149086070470000BB
:100EC0004004004090F83410C90706D001684A6811
:100ED000836B22F400321A434A6090F83410890779
:100EE00006D501684A68C36B22F480321A434A600F
:100EF00090F83410490706D501684A68036C22F45B
:100F000080221A434A6090F83410090706D5016818
:100F10004A68436C22F400421A434A6090F8341045
:100F2000C90606D501688A68836C22F480521A4388
:100F30008A6090F83410890606D501688A68C36C07
:100F400022F400521A438A6090F83410490611D5F1
:100F500001684A68036D22F480121A434A60016DE9
:100F6000B1F5801F06D101684A68436D22F4C002C2
:100F70001A434A6090F83410090606D501684A6899
:100F8000806D22F4002202434A607047F8B50025C4
:100F90000446C567FFF757F80746206800686FF0FA
:100FA0007E46000708D500223B464FF4001120463C
:100FB000009600F0FBFA60B92068006840070AD587
:100FC00000223B464FF480012046009600F0EEFAE6
:100FD00008B10320F8BD202084F8790084F87A0055
:100FE000002084F87850F8BD10B5806B0021A0F87F
:100FF0006A10A0F86210FFF78FFB10BD01680A6845
:1010000022F490720A6001688A6822F001028A6004
:10101000202180F87A10704710B5B0F86C2090F855
:101020007A300168222B05D0088B40F00800088335
:10103000022010BD898C8368B3F5805F01D10369FC
:101040006BB11140426E531C43661170B0F86A10C8
:10105000491E0904090CA0F86A1007D015E0436E78
:1010600011401980416E891C4166EFE701680A68EA
:1010700022F490720A6001688A6822F001028A6094
:10108000202180F87A10FEF7E3FF002010BD000059
:101090002DE9F04F044600688025FD4B0021D4F86F
:1010A00010C087B0A6680F46D4F81C8046EA0C062C
:1010B000D4F814C0A26A4CEA080C46EA0C06324383
:1010C0000668DFF8D0C306EA0C06164306602068FF
:1010D0004268E66822F44052324342602268A069C6
:1010E0009A4201D0266A3043A66AB6F1005F04D165
:1010F000D4E90B6C46EA0C0630439668DFF898C3D7
:1011000006EA0C06064396602068C26A666A22F008
:101110000F023243C262E14E2068E14AB04210D170
:10112000126802F03802182A74D005DCCAB3082A03
:101130007AD0102A47D179E0202A7BD0282A7CD186
:101140007AE0D84EB04209D1126802F00702062AAE
:1011500073D2DFE802F053696B6D6F71D24EB0420B
:1011600009D1126802F00702062A66D2DFE802F00F
:10117000465C5E606264CD4EB04209D1126802F0F6
:101180000702062A59D2DFE802F0394F515355576A
:10119000C74EB0420BD1126802F00702062A4CD2A9
:1011A00000E00EE0DFE802F02A4042444648C14E2B
:1011B000B04209D1126802F03802182A38D0BBDCDC
:1011C000B4E74FF0010538E0BB4EB04209D11268D8
:1011D00002F00702062A30D2DFE802F01026282AA1
:1011E0002C2EB64EB0420BD1126802F00702062A2E
:1011F00023D2DFE802F003191B1D1F2100251CE08C
:1012000098421AD1A64A121D126802F00702062A55
:1012100013D202E00CE007E00CE0DFE802F0030587
:1012200007090B0D022508E0042506E0402504E02F
:10123000082502E0102500E02025DFF864B2A04E6A
:101240009842DFF880A2ABF1540B73D1102D31D04E
:1012500006DC022D09D0042D0AD0082D2FD111E073
:10126000202D29D0402D2AD107E0FEF76BFF13E097
:101270006846FEF77DFF01980EE003A8FEF7F6FF33
:10128000049809E0DBF800105846890610D500687C
:10129000C0F3C1012AFA01F0002811D06168894623
:1012A00001EB410181420AD8B0EB093F07D808E0C1
:1012B0005046F3E78448F1E74FF40040EEE701279A
:1012C00033E1102D4FF000084ED006DC022D0FD078
:1012D000042D15D0082D04D12DE0202D4AD0402D0D
:1012E00013D00127794AA0F54071914270D9E6E701
:1012F000FEF728FF626A0023414636F812200DE00F
:101300006846FEF735FF019803E003A8FEF7AEFF3D
:1013100004980023616A36F811201946FEF79DFEF5
:1013200062680902030241EA10615008181841EB93
:10133000080115E032E0DBF800105846890609D5AF
:1013400000680023C0F3C1012AFA01F0616A36F88F
:10135000112015E0606A002336F8102050460FE097
:101360000023FEF77AFEBDE7606A002336F81020FE
:10137000554805E0606A002336F810204FF400401D
:101380000021FEF76AFE0902020241EA10614FEAFB
:10139000590010184A4641EB0801E1E7E3694FF4B0
:1013A000004293424DD1082D23D005DC8DB1012D93
:1013B00012D0042D06D112E0102D35D0202D3AD0B8
:1013C000402D11D0012721F00F00C1F34201084345
:1013D0005AE0FEF747FE16E0FEF749FE13E06846C6
:1013E000FEF7C6FE01980EE003A8FEF73FFF049843
:1013F00009E0DBF800105846890608D50068C0F3FC
:10140000C1012AFA01F0616A36F8111010E0606A31
:1014100036F81010BAFBF1F04100606801EB5001A2
:10142000B1FBF0F081B2CEE7606A36F810102648C2
:10143000B0FBF1F0F0E7606A36F81000B2FBF0F0B4
:10144000EAE7082D4AD00ADC0DB3012D43D0042D64
:101450007FF44DAF6846FEF78BFE019809E0102D32
:1014600052D0202D55D0402DF2D103A8FEF7FEFE1C
:101470000498616A36F81110B0FBF1F1606801EB75
:101480005001B1FBF0F080B22168C8604DE01FE070
:10149000000C0058F369FFCFFFF4FF11001001406A
:1014A000544402580044004000480040004C0040B2
:1014B000005000400014014000780040007C0040D3
:1014C000101600900090D00300093D00FFFC0F00B3
:1014D000FEF7C8FDCDE7FEF7CAFDCAE7DBF800203E
:1014E000594692060AD50968C1F3C1022AFA02F1E7
:1014F000626A36F81220B1FBF2F20FE0616A36F848
:101500001120BAFBF2F209E0616A36F811200949AC
:10151000F1E7616A36F81110B2FBF1F2616802EB93
:101520005102B2FBF1F189B2C16007B03846BDE8A3
:10153000F08F000000093D0090F87910212901D0BA
:1015400002207047B0F8621021B18168B1F5805F68
:1015500013D014E001680A68920004D58A6822F466
:1015600000028A6003E00A6822F080020A600068D4
:10157000016841F0400101600CE0016961B1C16D99
:101580004A1CC265026809781185B0F86210491ECC
:10159000A0F8621000207047C16D02680988C1F38D
:1015A00008011185C16D891CC165EEE72DE9F04187
:1015B0001E46174688460446069D1CE0681C1AD045
:1015C00025B1FEF740FD801BA84214D920680168B0
:1015D00021F4D07101602068816821F001018160EF
:1015E000202084F8790084F87A00002084F87800BC
:1015F0000320BDE8F0812068C16938EA010004D009
:101600000020B842DAD00020F3E70120F9E7FEE736
:10161000010002000400060008000A000C0010008F
:081620002000400080000001E1
:040000050800029954
:00000001FF
